:100000001EC18EC237C136C135C134C133C132C100
:1000100031C130C12FC12EC12DC12CC12BC12AC16C
:1000200029C128C127C10403090418037200610013
:10003000700068006E00650074002E006E006500A0
:1000400074000A033100300030003000050109055A
:10005000A1010901A10009300931150026FF007531
:100060000895028102C0050919012908150025011A
:10007000750195088102C005010902A1010901A1CC
:100080000005091901290215002501950275018154
:100090000295017506810305010930093115812595
:1000A0007F750895028106C0C012010101000000A1
:1000B000088117970A08010102030105010905A13A
:1000C000010901A10009300931150026FF0075085A
:1000D00095028102C0050919012904150025017541
:1000E0000195048102750195048103C0120101018B
:1000F000000000088117990A0801010000010501AC
:100100000905A1010901A10009300931150026FFE7
:1001100000750895028102C005091901290815001A
:100120002501750195088102C0120101010000003E
:10013000088117960A08010102030112010101005A
:1001400000000840177A05080101020301050109B2
:1001500005A1010901A10009300931150026FF00A0
:10016000750895028102C0050919012908150025A5
:1001700001750195088102C005010904A101090169
:10018000A100850109300931150026FF0075089589
:10019000028102050919012908150025017501953B
:1001A000088102C0C005010904A1010901A100855F
:1001B0000209300931150026FF00750895028102F9
:1001C0000509190129081500250175019508810205
:1001D000C0C005010904A1010901A100850309307E
:1001E0000931150026FF00750895028102050919DD
:1001F00001290815002501750195088102C0C00577
:10020000010904A1010901A1008504093009311582
:100210000026FF00750895028102050919012908C9
:1002200015002501750195088102C0C01201010168
:100230000000000881179D0A080101020301112432
:100240001FBECFE5D4E0DEBFCDBF11E0A0E6B0E039
:10025000E2E5FBE102C005900D92A438B107D9F7A1
:1002600012E0A4E8B1E001C01D92A431B107E1F7AA
:1002700037D36DCCC5CE85B7836085BF8BB780641F
:100280008BBF83EC8093EA0108950F931F93CF9364
:10029000DF939091FA0119160CF0A6C02091F70196
:1002A0008091F6018D3209F095C08AE58093610056
:1002B0009B3009F08FC0CCE0D0E0C21BD109C25006
:1002C000DE4F8881807609F077C01092E80189813D
:1002D000882351F41092E90188EE91E09093F9019E
:1002E0008093F80132E06BC0853021F48A818093DD
:1002F000FB0160C0863009F043C08B818130E1F1A1
:10030000823019F4CE016FD259C0833049F58A8109
:10031000882341F486E290E09093F9018093F801FC
:1003200034E050C0813041F48AE290E09093F901CA
:100330008093F80138E146C0823041F483E690E0D2
:100340009093F9018093F80134E239C08330C9F504
:1003500082E490E09093F9018093F8013CE032C090
:10036000813241F487E991E09093F9018093F8019B
:1003700039E028C0823229F5CE0135D2382F22C08B
:10038000883019F48DEF91E00AC0893021F48A8118
:100390008093FD010FC08A3041F488EE91E0909384
:1003A000F9018093F80131E00AC08B3019F483EC35
:1003B0008093EA0130E003C0CE0143D2382F20E819
:1003C00002C030E020EC8F81882339F48E818317BE
:1003D00028F003C080E020E801C0832F209384012F
:1003E000809360001092FA018091610084FF49C0FF
:1003F000809160008F3F09F444C0182F893008F0C5
:1004000018E0811B809360008091840180FD02C010
:100410000BE401C003EC8F5F809384012091F8010D
:100420003091F90186FD05C0D901912FE0EEF1E090
:1004300011C0A0EEB1E080E090E006C0F901E80F45
:10044000F91FE491ED9301961817C1F705C08D913E
:10045000819391509923D9F7F901E10FF11DF093A0
:10046000F901E093F80180EE91E0612F55D018304A
:1004700019F08FEF809360000093DF011C5F1093F1
:1004800061009AE080B3857031F49150D9F71092F1
:10049000FB011092F501DF91CF911F910F9108950B
:1004A0001F93DC01162F8091620084FF0AC08091A7
:1004B000EA0198E889278093EA01912FEBEEF1E0B9
:1004C00007C08AE580936200F8CF8D9181939150A7
:1004D0009923D9F78BEE91E0612F1ED01C5F10930A
:1004E00062001F910895A82FB92F8FEF9FEF41E071
:1004F00050EA615070F02D9138E0722F7827969570
:100500008795269570FF02C0842795273A95A9F70D
:10051000F0CF809590950895E6DF8D939D93089593
:10052000CF93CFB7CF93809BFECF809B09C0809B9A
:1005300007C0809B05C0809B03C0809B01C09EC0FC
:10054000DF93C091F701DD27C250DE4F809B02C0D0
:10055000DF91EBCF2F930F931F9300B32FEF00FB8F
:1005600020F94F933F9310B34FEF012700FB21F980
:100570003BE031C04E7F012F10B3216028C0102F07
:100580004D7F2260000000B329C04B7F2460012F03
:10059000000010B32BC010B3477F28602AC04F7EE5
:1005A00000B320612CC04F7D10B320622FC04F7B61
:1005B00000B3206432C0422700B349934FEF0000DC
:1005C000102710FB20F910B31570A9F1297F91F2C3
:1005D000012700FB21F900B3237F89F23150F0F1AC
:1005E000102710FB22F910B3277E79F2012700FBB8
:1005F00023F92F7C81F200B3102710FB24F92F7907
:1006000071F200C010B3012700FB25F92F7359F2D6
:1006100000C000B3102710FB26F9223040F200C0C2
:1006200010B3012700FB27F9243028F64F77206804
:1006300010B30000F9CF3B503195333010E41ABFAE
:10064000B8F0C31BD0400881033C41F10B3431F1B9
:100650001981412F1F772091F501121731F40936C6
:1006600091F10D3279F0013E69F022272093FC01CF
:100670003F914F911F910F912F91DF91CF91CFBF5C
:10068000CF9118950093FC013F914F911F910F91CD
:100690002F91DF91CAB7C6FD46CFF0CF0091FC0184
:1006A000002331F31091FA011123A1F53430A2F1A6
:1006B0003093FA010093F6011091F7013BE0311BF2
:1006C0003093F70129C00091FA0101301CF50AE5C9
:1006D00047FD09C03091610034FD20C000936100E6
:1006E000CFEDD1E01FC03091620034FD17C0009300
:1006F0006200CAEED1E016C0052710E002BB1FC0A1
:10070000052722C0052727C005272CC0052710E094
:1007100002BB33C04AE503C042ED01C0432FC4E130
:10072000D0E032E011B31560909A02B311BB5F9331
:1007300055E020E820FF052702BB279517951C3FB1
:10074000D8F620FF0527279502BB17951C3FC0F65A
:1007500020FF05272795179502BB1C3F98F620FF21
:100760000527279517951C3F02BB70F600C04991DD
:1007700020FF052702BB279517951C3F38F620FF61
:100780000527279502BB17951C3F38F520FF052745
:100790002795179502BB1C3F10F520FF05272795CD
:1007A00017951C3F02BBE8F4242F3A9519F60A7FEF
:1007B0005F9102BB00C01091FB01C651D04011F007
:1007C0001093F50110E41ABF016011B31A7F402F96
:1007D0004A7F02BB11BB42BB4BCF0527D3CF0527B6
:1007E000D8CF0527DDCFFC018081807641F581815E
:1007F000863029F583818230D1F0823269F08130F0
:10080000F1F48091890190918A019093F90180938C
:10081000F80180918B010895809186019091870164
:100820009093F9018093F80180918801089585E8FB
:1008300090E09093F9018093F80182E2089580E0BE
:100840000895DC012CE931E03093F9012093F8019F
:100850008C918076803209F041C011968C9111976D
:10086000823081F08A30F1F08130C1F5E0918C0165
:10087000F0918D010088F189E02DC90112966C91EB
:100880000995089512969C91892F8150883030F5F2
:10089000892F90E08D569E4F9093F9018093F80137
:1008A00081E008951296EC911297EE2359F4E4E951
:1008B000F1E013968C911397819381E0EC39F8075E
:1008C000C1F70CC08E2F8150883040F4F0E0ED5617
:1008D000FE4F13968C91808380E0089580E0089508
:1008E0006F927F928F929F92AF92BF92CF92DF9240
:1008F000EF92FF920F931F93DF93CF93CDB7DEB7A5
:10090000AA970FB6F894DEBF0FBECDBF88E0FE01F8
:100910003196DF01982F1D929A95E9F7E4E9F1E00D
:10092000DF011D928A95E9F7B89A87B3897F87BB63
:1009300088B3866088BBC09880E395E70197F1F79C
:1009400086B390E08670907095958795823091057A
:1009500009F43FC08330910509F43DC0019709F1C6
:10096000CAD6FC0190938D0180938C010284F3859B
:10097000E02D0995882309F452C0DE011996EBEEAB
:10098000F0E082E201900D928150E1F7A3E6B0E041
:10099000FE01399682E201900D928150E1F74CD828
:1009A0003AC04CD790938D0180938C01DE0119964B
:1009B000E9ECF0E082E201900D928150E1F7A3E6CC
:1009C000B0E0FE01399682E201900D928150E1F78C
:1009D00026C031D420C052D1FC0190938D01809368
:1009E0008C010284F385E02D0995ECD18823B9F0C0
:1009F000DE011996E7EAF0E082E201900D92815063
:100A0000E1F7A3E6B0E0FE01399682E201900D9293
:100A10008150E1F798D390938D0180938C01E09100
:100A20008C01F0918D018481958190938701809351
:100A3000860182818093880180859185009731F0BD
:100A400090938A0180938901868107C089E291E0B1
:100A500090938A018093890180D680938B01809145
:100A6000880180939E0014BA8FEF85BB88EF82BB0C
:100A700085E081BB11BA83BF8FE085BD84EC83BD67
:100A800085B78F7885BFE0918C01F0918D0102844C
:100A9000F385E02D0995EFDB7894FF2411E06624BF
:100AA00063944E010894811C911C21E0C22ED12C2C
:100AB00090E8792E8CE2A82E81E0B82E02C0FF24A7
:100AC00010E0A895E2DB112341F0E0918C01F09158
:100AD0008D010484F585E02D099508B600FE27C038
:100AE00068BE40918C0150918D01D40120E030E02E
:100AF00018C0F901EC56FE4FE081EE2379F08C919D
:100B0000853018F085508C9309C0EC93C601022EF5
:100B100002C0880F991F0A94E2F7F82A2F5F3F4F0F
:100B20001196FA01808191812817390714F308B6CC
:100B300007FE31C078BE85B7806885BF889585B7C8
:100B40008F7785BFC5010197F1F7E0918C01F09196
:100B50008D010484F585E02D099500E010E012C0B8
:100B60000684F785E02D802F8F5F0995882341F05B
:100B7000C601002E02C0880F991F0A94E2F7F82AD6
:100B80000F5F1F4FE0918C01F0918D018081918169
:100B9000081719072CF3FF2009F492CF00E010E0AA
:100BA000EF2CFF24E7FCF09422C0C701002E02C006
:100BB000959587950A94E2F780FF17C080916200AF
:100BC00084FF13C0602F6F5F0088F189E02D8EE8ED
:100BD00091E00995682F8EE891E062DC02C055DB58
:100BE000A8958091620084FFFACF0F5F1F4FE091BC
:100BF0008C01F0918D018081918108171907ACF269
:100C00005ECFAC9A80E38A95F1F7AC9880E090E0F3
:100C100030E048E1242F2A95F1F7AD98330F9B9BE4
:100C20003160242F2A95F1F7AD9A0196883091050D
:100C300089F73093A30180E090E048E1242F2A95C2
:100C4000F1F7AD9836959B9B3068242F2A95F1F7E4
:100C5000AD9A01968830910589F73093A4010895E3
:100C60001F931FB7F894A49AA59AA398AB9AAD9A2C
:100C7000AC98C7DF1FBF80E01F9108958CE490E01F
:100C800090931201809311018DE091E00895FC0191
:100C9000009709F453C0A091A3018091A401682F8B
:100CA00070E0CB01807F9070803F910521F481E05E
:100CB0008093A20102C01092A2014A2F50E0A0FD31
:100CC00003C020E830E002C02FEF30E041FF02C057
:100CD00020E030E042FD03C080E890E002C08FEFEA
:100CE00090E043FF02C080E090E020838183CA014E
:100CF0008074907025E0959587952A95E1F79A0183
:100D000020723070B3E035952795BA95E1F7982FAA
:100D1000922BAA1FAA27AA1F9A2B40715070559593
:100D20004795942B92838091A201882339F484E023
:100D3000660F771F8A95E1F7962B92838091A30126
:100D40009091A4019093A6018093A50183E008955A
:100D500080911F0190912001892B31F01092200188
:100D600010921F0181E0089583EA91E065EA71E045
:100D700042E050E0DFD60895FC01AC9A80E38A950A
:100D8000F1F7AC9890E028E1822F8A95F1F7AD98C1
:100D9000822F8A95F1F7AD9A9F5F9830A9F79081DD
:100DA00020E038E1832F8A95F1F7AD98990F9B9B4E
:100DB0009160832F8A95F1F7AD9A2F5F283091F7D4
:100DC00090830895DF93CF930F92CDB7DEB7CE0116
:100DD0000196D2DF90E089818F70813009F491E033
:100DE000892F0F90CF91DF9108956F927F928F920C
:100DF0009F92AF92BF92CF92DF92EF92FF920F93AA
:100E00001F93DF93CF930F92CDB7DEB773E0E72E3A
:100E1000F12CE822F92206E010E04E010894811C32
:100E2000911C68EBA62E6BE0B62E54E0752E40E3C5
:100E3000642E30E8C32E3BEBD32EC4019DDF8981A5
:100E400090E08073907024E0959587952A95E1F75E
:100E50008E159F0529F4F092B001E092AF011CC0FD
:100E6000C5010197F1F780E090E0AC9A272D2A9513
:100E7000F1F7AD98AD9A272D2A95F1F7AC98262D6C
:100E80002A95F1F701968F31910579F7C6010197FF
:100E9000F1F70150104089F60F90CF91DF911F912B
:100EA0000F91FF90EF90DF90CF90BF90AF909F9009
:100EB0008F907F906F900895DF93CF930F92CDB76F
:100EC000DEB7CE01019658DF2981822F8F708130E5
:100ED00079F58091AD019091AE01892B71F5229544
:100EE000269526952370822F90E08130910571F030
:100EF000823091051CF4892B79F013C08230910562
:100F000041F0039771F480E090E00AC081E090E046
:100F100007C082E090E069DF8091AF019091B0015D
:100F200064DFCE01019628DF89818F70813029F03E
:100F30001092AE011092AD0156C081E090E0909306
:100F4000AE018093AD0189818093B10180E797E183
:100F50000197F1F78CED95E00197F1F780E090E0D3
:100F600050E030E2232F2A95F1F7AD98550F9B9B67
:100F700051600000AD9A01968830910599F780E0A4
:100F800090E030E040E2242F2A95F1F7AD98330F3E
:100F90009B9B31600000AD9A01968830910599F7CE
:100FA000232F2F77452F4F7737FD219557FD4195FB
:100FB000332727FD30958091A7019091A801820FDA
:100FC000931F9093A8018093A701242F332727FD17
:100FD00030958091A9019091AA01820F931F90935F
:100FE000AA018093A9010F90CF91DF910895A49A4F
:100FF000A59AA398AB9AAD9AAC985EDF8091B101A7
:10100000829586958695837090E08130910571F088
:10101000823091051CF4892B31F00EC0823091058D
:1010200041F0039749F480E090E005C081E090E052
:1010300002C082E090E0D9DE80E008958091330123
:1010400090913401892B29F01092340110923301D0
:101050001DC09091B1018091B2019817B9F420910F
:10106000A7013091A8018091B3019091B401281794
:10107000390761F440E02091A9013091AA018091E3
:10108000B5019091B6012817390709F041E0842F86
:101090000895FC01009709F454C08091AB01909130
:1010A000AC01892B41F01082118212821092AC01A6
:1010B0001092AB0146C0A091B1018A2F829586950E
:1010C0008695837080836091A7017091A8018FEF4E
:1010D0006138780714F481E806C06038710514F0AF
:1010E0008FE701C0862F4091A9015091AA019FEF7F
:1010F0004138590714F421E806C04038510514F06E
:101100002FE701C0242F81832283992787FD9095A3
:101110009093B4018093B301332727FD309530932A
:10112000B6012093B501A093B201681B790B7093AF
:10113000A8016093A701421B530B5093AA0140934F
:10114000A90183E0089587E790E0909326018093BA
:10115000250189EA90E090932A018093290181E298
:1011600091E00895A49AA59AA398AB9AAD9AAC98E9
:1011700080E00895AC9A80E38A95F1F7AC9880E01E
:1011800090E030E048E1242F2A95F1F7AD98330F35
:101190009B9B3160242F2A95F1F7AD9A01968830F8
:1011A000910589F73093B70108958091B701909127
:1011B000B801891B0895FC010097B9F16091B7014E
:1011C000462F50E060FD03C020E830E002C02FEF62
:1011D00030E041FF02C020E030E042FD03C080E883
:1011E00090E002C08FEF90E043FF02C080E090E00B
:1011F000208381839A012074307075E0359527959E
:101200007A95E1F7CA018072907033E095958795E1
:101210003A95E1F7282B661F6627661F262B40713B
:10122000507055954795242B22838091B701809368
:10123000B80183E008958BEB90E090933A0180939E
:1012400039018CEE90E090933E0180933D0185E35F
:1012500091E0089523B366B330E0A9014071507066
:10126000A3E055954795AA95E1F7C901887090705C
:1012700095958795482B862F8072482BC9018470DD
:101280009070880F991F482BC9018270907073E08D
:10129000880F991F7A95E1F7482B2072307055E03E
:1012A000359527955A95E1F7422B80915B01843063
:1012B00011F0842F0895862F90E080719070880F30
:1012C000991F880F991F842B0895DF92EF92FF9248
:1012D0000F931F93CF93DF93EC01A89A00E5802F23
:1012E0008A95F1F7B7DFD82E80915B01823028F420
:1012F000D8828FEF89838A8329C0A898802F8A9506
:10130000F1F7A8DFF82EA89A802F8A95F1F7A89810
:10131000802F8A95F1F79EDFE82EA89A802F8A9574
:10132000F1F7A898802F8A95F1F794DF182FA89AE3
:10133000802F8A95F1F78EDFA898902F9A95F1F774
:10134000A89AD882F9828A83EB821C83DF91CF919D
:101350001F910F91FF90EF90DF900895DF92EF9231
:10136000FF920F931F93CF93DF9300E010E0C0E054
:10137000D0E0EE24FF24B8E2DB2E6CDF85FF04C052
:101380000894E11CF11C01C021968D2D8A95F1F77E
:101390000F5F1F4F0436110581F7A2971CF420E060
:1013A00030E009C080E090E022E2E216F10414F09F
:1013B00081E090E09C01C901DF91CF911F910F91D5
:1013C000FF90EF90DF9008957F928F929F92AF925F
:1013D000BF92CF92DF92EF92FF920F931F93DF9312
:1013E000CF9300D000D00F92CDB7DEB710915B0144
:1013F000143009F07FC01091B90110FD07C0CC2452
:10140000DD24E1E0F0E0AA24BB2408C021E0C22EE4
:10141000D12CE0E0F0E091E0A92EB12CE554FE4F94
:1014200080E880831092BD0115DF282F30E084FD15
:1014300005C08091BD0181608093BD01C9018074A8
:10144000907011FF10C0892B29F48091BD0182603A
:101450008093BD01EE24FF2484E0782E08EF802ED7
:1014600018E0912E44C0892BA9F78091BD018160BD
:10147000EFCFF0DE85FD08C0972D9A95F1F70F5F4D
:101480001F4F04361105A9F785FF26C0E3DE182F8C
:10149000892D8A95F1F7DEDE85FF21C0882D8A959A
:1014A000F1F7D8DE85FD1BC0012F0295007FD2DE4B
:1014B000182F1F70892D8A95F1F7CCDE85FD0FC09E
:1014C000802F812BAB2809F080952BEB31E0C20EE9
:1014D000D31EF60180837CC0882D8A95F1F708948D
:1014E000E11CF11CF4E0EF16F10409F471C000E016
:1014F00010E0BFCFCE010196E8DE998190958A81F8
:1015000080958A836B81609590FD03C040E850E030
:1015100002C040E050E091FF02C04FEF50E092FD6A
:1015200003C020E830E002C020E030E093FF02C0BA
:101530002FEF30E02093BB014093BC011092BD011E
:101540001230D0F18A81282F84FF03C081E080937C
:10155000BD0194FF05C08091BD0182608093BD01F3
:1015600095FF05C08091BD0184608093BD0125FF7A
:1015700005C08091BD0188608093BD01133041F5A5
:10158000962F62FF05C08091BD0180618093BD01EF
:1015900091FF05C08091BD0180628093BD0190FFE5
:1015A00005C08091BD0180648093BD0193FF10C090
:1015B0008091BD0180680AC094FF03C081E08093E0
:1015C000BD0195FF05C08091BD0182608093BD0182
:1015D0000F900F900F900F900F90CF91DF911F9170
:1015E0000F91FF90EF90DF90CF90BF90AF909F90C2
:1015F0008F907F9008951F93DF93CF9300D000D0FA
:101600000F92CDB7DEB71FB7F894B99AC19887B3D8
:101610008F7C87BB88B3806388BBA09AA89A84B369
:10162000817C84BB85B38E6385BB88EE93E02CE21E
:1016300031E0F9013197F1F70197D9F78FDE892B66
:1016400029F184E080935B0182E090E09093BA01FD
:101650008093B901B9DE1092BA011092B90180915C
:10166000BD01282F80FF06C081E090E09093BA0171
:101670008093B90121FF34C08091B9019091BA01E2
:1016800082609093BA018093B9012AC0CE0101967D
:101690001CDE81E080935B01898190E08F70907007
:1016A0008330910519F41FBF8FEF1CC00F9789F489
:1016B0008A818F70833069F48C818F70833021F43C
:1016C0008D818F70833011F083E001C082E08093C0
:1016D0005B018A8185FD03C083E080935B0174DE3A
:1016E0001FBF80E00F900F900F900F900F90CF9141
:1016F000DF911F9108958EEF90E090934C018093BD
:101700004B0187E491E00895009741F0DC01EBEB99
:10171000F1E083E001900D928150E1F7AEEBB1E092
:10172000EBEBF1E083E001900D928150E1F783E073
:1017300008958091590190915A01892B31F01092AE
:101740005A011092590181E008958BEB91E06EEB04
:1017500071E043E050E0EED1089582E190E0089519
:10176000A89888EB9BE0FC013197F1F7A99AFC015E
:101770003197F1F723B3A9980197F1F783B3A89AAA
:1017800090E08C739070880F991F880F991F30E03C
:101790002C7330703595279535952795822B80953C
:1017A000982F83FD03C040E850E002C040E050E0C5
:1017B00091FF02C04FEF50E090FD03C020E830E001
:1017C00002C020E030E092FF02C02FEF30E0209313
:1017D000C1014093C2011092C30187FF03C081E0A1
:1017E0008093C30196FF05C08091C30182608093FE
:1017F000C30195FF05C08091C30184608093C3013C
:1018000094FF05C08091C30188608093C30108954F
:101810001F931FB7F894B99AC19884B3837C84BB93
:1018200085B38C6385BB85B3836085BB84B38360DC
:1018300084BB96DF1FBF80E01F9108958DE491E087
:1018400090936101809360018BE391E09093650137
:10185000809364018CE591E00895009741F0DC01EC
:10186000E1ECF1E083E001900D928150E1F7A4EC0E
:10187000B1E0E1ECF1E083E001900D928150E1F7FD
:1018800083E0089580916E0190916F01892B31F072
:1018900010926F0110926E0181E0089581EC91E049
:1018A00064EC71E043E050E045D108958FB7F894BF
:1018B000B99AC198BD9AC59AA09AA89A94B3917CF6
:1018C00094BB95B39E6395BB8FBF80E008958F92C4
:1018D0009F92AF92BF92CF92DF92EF92FF920F93BF
:1018E0001F93DF93CF93CDB7DEB762970FB6F8940F
:1018F000DEBF0FBECDBFA8988CE291E00197F1F753
:1019000060E070E08E010F5F1F4F9FE0F92EACE2A8
:10191000B1E060FF04C0C59A999BFECF03C0C59893
:101920009999FECF43B350E09A01287030703595F5
:101930002795CA0180719070F3E095958795FA9587
:10194000E1F7282BCA0184709070880F991F282B0B
:101950004072507035E0559547953A95E1F7242B44
:10196000F801E60FF71F2F252083CD010197F1F72E
:101970006F5F7F4F6231710561F6C59AA89A8981C0
:101980008F3009F046C08A818F3009F042C093E061
:10199000E92EF12CEC0EFD1E26E030E0CC24DD24F7
:1019A0004E010894811C911C87E0A82EB12CAC0E2E
:1019B000BD1ED7018C918E3019F08F3021F406C0F6
:1019C00063E070E005C060E070E002C062E070E0DB
:1019D0008401020F131FF601E953FE4F40E050E06F
:1019E00006C0D8018D918D0181934F5F5F4FDA0161
:1019F000A20FB31F46175707A4F30894E11CF11C6C
:101A0000E3E0F0E0CE0EDF1EEA14FB0411F09D01CE
:101A1000D0CF62960FB6F894DEBF0FBECDBFCF9188
:101A2000DF911F910F91FF90EF90DF90CF90BF90CB
:101A3000AF909F908F90089588E791E09093750103
:101A4000809374018CE292E0909379018093780105
:101A500080E791E008950F931F93CF93DF938C015C
:101A6000662311F480E046C0862F992787FD909564
:101A700001979C01220F331F280F391FE901C95319
:101A8000DE4FD901AD52BE4FFE0183E001900D92B1
:101A90008150E1F7888180FD03C040E850E002C03A
:101AA00040E050E081FF02C04FEF50E082FD03C0F4
:101AB00020E830E002C020E030E083FF02C02FEFDA
:101AC00030E0898190E080FD92E081FD946082FDAC
:101AD000916083FD98608A8180FD906481FD9062B1
:101AE00082FD906183FD9068F801608321834283C9
:101AF000938384E0DF91CF911F910F910895282F58
:101B00008091820190918301892B31F010928301A1
:101B10001092820181E00895215063E02602B00115
:101B20001124CB0189539E4F6D527E4F43E050E00C
:101B300001D00895FB01DC0104C08D910190801952
:101B400021F441505040C8F7881B990B0895F89430
:021B5000FFCFC5
:101B5200FF5A5A22032800530029004E0045005321
:101B6200002F00410074006100720069005F00559F
:101B720000530042000902220001010080320904E0
:101B82000000010300000009210101000122000000
:101B92000705810308000A220353004E0045005343
:101BA200004D006F007500730065005F0074006FE8
:101BB200005F0055005300420022034E006500639F
:101BC200002D0050006300200065006E0067006970
:101BD200006E0065002000200020002203530065F3
:101BE20000670061004D0075006C007400690074AC
:101BF20000610070005F0055005300420001002B9D
:101C02000000000000000030060106A80647060199
:101C12000001003200000012000000F7075C071EFE
:101C2200084908010001003100000012000000B262
:101C320008BA08D508DB0801002B000000000000EC
:101C420000FB0AE409990B840B01000201002B003E
:101C5200000012000000080CB00B420C2D0C010019
:101C62000400B400000012000000560C670C7F0D47
:041C72002B0D010035
:00000001FF
